:020000040000FA
:06000000E0EF07F0120022
:0600080004EF08F01200F5
:060018000CEF08F01200DD
:0E0020000100EC0F0000FE03000002000000D3
:02002E00F00ED2
:100030008C1695160001636B676968696969666B60
:10004000010E6A6F1200D9CFE6FFE1CFD9FFE65269
:10005000000163511FE1040108BF1BD0400EE66E92
:10006000700EE66E030EE66E11EC06F0E552E552F8
:10007000E5520001010E636FDF6A400EDF5C09E2AA
:10008000DF50EA6AB00FE96E030EEA22EF6ADF2A58
:10009000F4D781D103017051080A01E16BD10F0A35
:1000A00001E119D1010A01E10ED1030A01E1AAD04F
:1000B000010A6AE0070A5DE0010A01E06CD1030170
:1000C000020EB06F03013A0EB16F0301010EB26F61
:1000D0000301010EB36F0301B46B100EB56FB66B65
:1000E000B76B0301B86B700EB96FBA6BBB6B0301D2
:1000F000030EBC6F0301BD6BBE6B300EBF6FC06BD8
:1001000003010C0EC16FC26BC36BC46B0301010E04
:10011000C56F0301C66BC76B200EC86FC96B0301A7
:10012000080ECA6FCB6BCC6BCD6B0301CE6903019C
:10013000020ECE6F0301CF6BD06BF00ED16FD26B7E
:100140000301D36B010ED46FD56BD66B0301D76956
:1001500004010CBF0DD0400EE66EB00EE66E030E2D
:10016000E66EE1EC05F0E552E552E5520001636B05
:1001700012D10001010E6A6F0301715102E1000109
:100180006A6B0001636B07D1400E0001646F656B01
:100190000001000E645D020E65591FE2040064C098
:1001A00000F065C001F0026A060E1F0B00C0F6FFEA
:1001B00001C0F7FF02C0F8FF06E0D890F636F73628
:1001C000F836E806FAE1940EA66E9ED972EC06F0B7
:1001D0000001642B000E6523DBD7DF6ADF50A96EB8
:1001E000A868040EA66E72EC06F08ED9DF2AF6E13E
:1001F000F66AF76A200EF86E940EA66E85D9000195
:10020000636BC9D0300E0301735D07E100016A51D1
:1002100001E130D90001636BBED0F00E0301735DC4
:1002200004E150D90001636BB6D0E868000167199A
:1002300005E1E868681902E1E868691906E171C337
:1002400067F072C368F073C369F0670EE96E000E61
:10025000EA6EEE500301711908E1EE5003017219C4
:1002600004E1EE500301731900E12AE1DF6A0301A2
:100270007551DF5C25E23A0E0301D8807555DF2405
:10028000EA6A760FE96E030EEA22EF50E66E00018D
:100290006651EA6A6B0FE96E000EEA22E552E750FA
:1002A000EF6E0001662B0001672B000E6823000E25
:1002B0006923200E0001665D01E172D8DF2AD7D7DD
:1002C0000001636B68D06CD800016769686969696F
:1002D0000001636B60D00301070EB06F71C3B1F30F
:1002E00072C3B2F373C3B3F374C3B4F375C3B5F39A
:1002F00071C3F6FF72C3F7FF73C3F8FFDF6A030130
:100300007551DF5C26E2F00E0301735D13E1DF50EF
:1003100003017125A96EA66AA6803A0E0301D88052
:100320007555DF24EA6AB60FE96E030EEA22A8CFFC
:10033000EFFF0DD009003A0E0301D8807555DF2478
:10034000EA6AB60FE96E030EEA22F5CFEFFFDF2A65
:10035000D6D704010CBF0DD0400EE66EB00EE66E8F
:10036000030EE66EE1EC05F0E552E552E5520001C0
:10037000636B11D06D926D6ADF6AFF0EDF5C09E27C
:10038000E868E85004E0E80600D000D0FAD7DF2A99
:10039000F4D7FF0000D0E552E552E7CFD9FF1200B5
:1003A000D9CFE6FFE1CFD9FF030EE126010EDB6ACC
:1003B00066C000F0016A026A00500001675DF66ED7
:1003C000015000016859F76E025000016959F86E3A
:1003D0001F0EF614E76E020EE7CFDBFFE00EF616F7
:1003E000DF6A200EDF5C1EE2020EDB5015E1000129
:1003F00066510FE0010EDB50EA6A6B0FE96E000EEA
:10040000EA22EF50F56E0D00010EDB2A00016607AF
:1004100002D0F5680D0004D0F5680D00020EDB0671
:10042000DF2ADFD70A00A40EA66E6ED8DF6A0001AD
:100430006651DF5C15E2010EDB50DF24EA6A6B0FC8
:10044000E96E000EEA22EF50E66EDF50EA6A6B0FAB
:10045000E96E000EEA22E552E750EF6EDF2AE7D799
:10046000030EE15C02E2E16AE552E16EE552E7CF9C
:10047000D9FF1200D9CFE6FFE1CFD9FFE65271C311
:10048000F6FF72C3F7FF73C3F8FFDF6A030175510C
:10049000DF5C13E23A0E0301D8807555DF24EA6A67
:1004A000760FE96E030EEA22EF50F56E0C00C40ED3
:1004B000A66E2AD80900DF2AE9D7E552E552E7CF30
:1004C000D9FF1200D9CFE6FFE1CFD9FFE652DF6AAC
:1004D00003017551DF5C13E2DF507125A96E3A0EFE
:1004E000D8807555DF24EA6A760FE96E030EEA229A
:1004F000EF50A86E040EA66E07D8DF2AE9D7E552A2
:10050000E552E7CFD9FF1200F29E550EA76EAA0E54
:0C051000A76EA682A6B2FED7A694120029
:04051C006C500CE132
:100520006896040100513C0BE842E8420D0802E1E4
:100530000AD8010C3BD8010C040E6C5C03E16896F0
:1005400044D8010C000C70D9E652040104BF046BBE
:100550000001B36BAB6BAC6BB16BB26B25EC04F011
:10056000DF6ADF50006E016A010E005C000E015868
:100570001AE20001AC5117E1F76ADF34FE0BF736DF
:10058000F66E9C0EF6260E0EF7220900F5CF00F04F
:100590000800F5CF01F004D001C0FAFF0050F96E59
:1005A000FBDFDF2ADED7ACD8E55243D1020E0001D3
:1005B000AB5D09E179D8040100BD02D0C80E01D0BD
:1005C000880E006F1200B9EF03F0040E0301FA5D0C
:1005D00009E112C46EFF6E50000802E2050E01D060
:1005E000030EFA6F0001AB0510E111D8020E0001F5
:1005F000B35D03E10401840E06D0040104BD02D002
:10060000C80E01D0880E046F1200B9EF03F00CD9A8
:10061000020EE1260001080EB15D000EB2590DE296
:10062000B1C0DEFFB2C0DDFFB35102E1010E03D065
:10063000B30506E1020EB36F03D0080EDE6EDD6A6D
:10064000040104930491010EDB500413DFCF05F481
:10065000000EDB500001B15F010EDB50B25B180EE3
:10066000AF6F040EB06F0301FBA30CD0D6D815E01A
:10067000ADC0F6FFAEC0F7FF0800F550BED8F6E2F9
:10068000DB06F4D7CAD809E0ADC0E9FFAEC0EAFF87
:10069000EF50B3D8F7E2DB06F5D7020EE15C02E2D9
:1006A000E16AE552E16EC5D0BFD8020EE126030E25
:1006B00004010015E76E010EE7CFDBFF01C4DFFF89
:1006C000DE500001B127DD50B223180EAD6F040ECD
:1006D000AE6FA3D80EE0ADC0E9FFAEC0EAFFEF50A9
:1006E000AFC0E9FFB0C0EAFFEF6EA7D8F2E2DB06C9
:1006F000F0D7020EE15C02E2E16AE552E16E99D0C8
:100700006D980001AC5105E180D8840E006F0401A2
:100710001DD0040110AF1CD00001B1510401165DC1
:100720000001B2510401175904E216C4B1F017C414
:10073000B2F06DDF0001010EAB6F67D8800E006F65
:100740000401180E066F040E076FC80E046F120026
:100750000001020EAB6F0401056BC80E046F0401AB
:10076000080E016F180E026F040E036FC80E006FA3
:1007700012005AD8E652020E0001AB5D35E16D5011
:10078000100B32E004010151006E016A080E0018DE
:100790002BE1015029E100513C0BE842E8420D08F1
:1007A00023E10051800B20E1100E026F040E036F55
:1007B000DF6ADF50006E016A080E005C000E01580F
:1007C0001AE2DF50EA6A180FE96E040EEA22EF50CF
:1007D000E66EDF50EA6A100FE96E040EEA22E55277
:1007E000E750EF6EDF2AE5D70001AB6B0ED88C0E19
:1007F000006F0401046BE5521CD0AFC0E9FFB0C02C
:10080000EAFFEF6E00011DEF04F00401080E016F16
:10081000100E026F040E036F1200D9CFE9FFDACF7A
:10082000EAFFEE50ED101200D9CFE6FFE1CFD9FF7D
:100830001200E552E7CFD9FF1200AF2B000EB02314
:0A084000AD2BAE23DF06010E1200FF
:06084A0004011051600BD7
:10085000E842E842E842E842E842000901E01200CA
:100860001151070A40E00B0A3EE0070A33E0010A93
:1008700023E00B0A1FE0020A1DE0030A19E0080A40
:1008800010E0010A0CE00F0A08E0030A01E0120080
:1008900012D90301040EFA6F120074EF04F0ABEFEB
:1008A00004F009D90001FC0EAD6F030EAE6F0CD041
:1008B000C6EF04F0F8EF04F002D90001AD6FAE6BA3
:1008C000FD0EAD27030EAE230301FB930001010EC5
:1008D000B16F1200F4D8EA6AFD0FE96E030EEA2246
:1008E00012C4EFFF12001200800E0401105D32E10D
:1008F0001351030A1FE0010A0AE0030A29E1DBD8C9
:100900000001DC0EAD6F0D0EAE6F120E1ED0B2D810
:10091000920EF6260E0EC0D8020E0001F76AAD2523
:10092000F66EAE51F7220900F5CFB1F00A00F5CF0F
:10093000B2F00ED09FD8960EF6260E0EADD8ADC0F2
:10094000F6FFAEC0F7FF0800F5500001B16FB26BC3
:100950000301FB831200AFD80F0EE66E710EE66E38
:100960000F0EA2D8010EE66EFD0EE66E030E9CD8A9
:1009700012C4FCF30401125104E10301050EFA6FE5
:1009800012000301060EFA6FCCEF05F00401186B9C
:10099000196B040110511F0B020A0FE0030A0BE050
:1009A000010A18E188D8040118810301FBA112D0C3
:1009B000040118830FD07FD80DD050D801E0010E6C
:1009C00062D8AFC0E9FFEA6EEF50040B03E0040108
:1009D000010E186F0001AC050AE10001180EAD6FA1
:1009E000040EAE6F0301FB930001020EB16F120003
:1009F000040112050EE110511F0B00090AE15BD83A
:100A0000030E0401115D03E10301FB8102D0030128
:100A1000FB910401125121E110511F0B02081DE14D
:100A200014510F0B000919E019D801E0010E2BD861
:100A3000030E0401115D02E1840E03D014AF07D050
:100A4000400EAFC0E9FFB0C0EAFFEF6E1200880EA3
:100A5000AFC0E9FFB0C0EAFFEF6E120030D80F0B55
:100A6000080DF350016A000F006E040E01221451AC
:100A7000800B120020D804011251F66EF76AD8904C
:100A8000F636F7361200040DF35000010024AF6F64
:100A9000000E0120B06F1200F7220900F5CFADF073
:100AA0000A00F5CFAEF01200E66ED9EC06F0E55282
:100AB000E552E55212000001010EAC6F1200FBDF9F
:060AC000040114511200B4
:0A0AC600040110511F0B010801E0AC
:100AD0001200145101E01200060E115D24E11351C1
:100AE000230A1FE0010A0DE0030A1BE1DBD8030122
:100AF000FC0505E10001000EAD6F0E0EAE6F090E94
:100B00000DD0D0D80301FC0505E10001750EAD6FD5
:100B10000E0EAE6F0301FC0504E11D0E0001B16F66
:100B2000B26B0301FB8304011051600BE842E84201
:100B3000E842E842E842010801E0120011510B0AC4
:100B400025E0080A17E0090A11E0080A09E00B0A83
:100B500005E0080A01E01200CAEF05F0CBEF05F04E
:100B6000A1D80001B40EAD6F000E09D09BD813C4FC
:100B7000B4F0120097D80001B50EAD6F000EAE6F45
:100B80000301FB930001010EB16F12008BD812C458
:100B9000B5F01200120012000001B66B1E0E716E4D
:100BA0000401400E096F200E0A6F040E0B6F880EB1
:100BB000086F0401600E0E6F040E0F6F400E0C6F75
:100BC0001200D9CFE6FFE1CFD9FFE652FC0EDB5091
:100BD000400805E2400EF36EFC0EF3CFDBFFDF6A48
:100BE000FC0EDB50DF5C0FE2DF5050D8EF50E66EBA
:100BF000DF50EA6A600FE96E040EEA22E552E75020
:100C0000EF6EDF2AEDD7FC0EDBCF0DF4400E0401B2
:100C10000C170C7D880E0C13E552E552E7CFD9FF77
:100C20001200D9CFE6FFE1CFD9FF0001B66B040176
:100C300008BF26D0FC0EDBCF00F00951D88000544D
:100C400003E2FC0E09C4DBFF0001B66BFC0EDB50B7
:100C5000B65D0FE2B651EA6A200FE96E040EEA2291
:100C6000EF50E66EB65112D8E552E750EF6EB62B54
:100C7000EDD70401400E096F0817087D880E081390
:100C80000001B651E552E7CFD9FF1200E76EFD0E25
:100C9000DBCFE9FFFE0EDBCFEAFFE750E926000ECF
:0C0CA000EA2212000001020EAC6F1200EC
:040CAC006DA60CD84D
:100CB0000301FA0508E16DBA06D0686A696A6980BD
:100CC0006988020EFA6F12006D6A696A6D86030107
:100CD000010EFA6F12006D6A696A0301FA6B120065
:100CE0006BEF06F00301FA5101E1120068B425D858
:100CF0006DB2120068B038D868B817D868BA24D86E
:100D0000030E0301FA5D01E212000001B76B040E4D
:100D1000B75D0AE268A608D08EEC02F0000901E196
:100D200068960001B72BF3D71200698468986D822A
:100D3000A19AA08A0300A09A12006D92699468A4F7
:100D400002D06894FCD7120070A00CD0800E040171
:100D5000005D07E1840E0401045D03E104018C0ED3
:100D6000006F7090689A12006A6A686A9F0E6B6ED4
:100D70007B0E696E6E6A0F0EE66E710EE66E0F0EDA
:100D8000E66E17D8E552E552E552160E706E68A66B
:100D900005D0689600D000D00000F9D76D98B9EC66
:100DA00003F00301FB910301FC6B0301030EFA6FD7
:100DB0001200D9CFE6FFE1CFD9FFFD0EDBCFE9FF6F
:100DC000FE0EDBCFEAFFFC0EDB5004E0EE6AFC0E09
:0C0DD000DB06F9D7E552E7CFD9FF12008F
:040DDC0012010002FE
:100DE00000000008D8043C000200010200010902D2
:100DF0002900010100C032090400000203000000C4
:100E0000092111010001221D000705810340000195
:100E1000070501034000010403090434034D006980
:100E200000630072006F00630068006900700020BA
:100E30000054006500630068006E006F006C006F76
:100E40000067007900200049006E0063002E002634
:100E50000348004900440020005500530042002090
:100E60000042006F006F0074006C006F006100644E
:100E700000650072000600FF0901A1011901294067
:100E8000150026FF0075089540810219012940913F
:0E0E900002C0EE0DEE0D170E1B0E4F0EC60A21
:020E9E00200E24
:100EA000F66E000EF76E000EF86E03010900F550A5
:100EB000F56F0900F550F66F03E1F56701D03DD0FD
:100EC0000900F550F06F0900F550F16F0900F55079
:100ED000F26F09000900F550E96E0900F550EA6E5D
:100EE000090009000900F550F36F0900F550F46F8F
:100EF00009000900F6CFF7F3F7CFF8F3F8CFF9F3CD
:100F0000F0C3F6FFF1C3F7FFF2C3F8FF0301F35399
:100F100002E1F45307E00900F550EE6EF307F8E242
:100F2000F407F9D7F7C3F6FFF8C3F7FFF9C3F8FFE3
:0C0F30000301F507000EF65BBFD71200AE
:040F3C000F0EC16E65
:100F400081A804D0070EC16E00EF08F00ED804008F
:100F500016D819D8060E0301FA5D05E16D50020B93
:100F600002E123EC00F0F3D71200140E6F6E0301C0
:100F7000FA6B0301FB6B0301FC6B17EF00F056ECFF
:100F800006F072EF06F00301FE51FF1104E1100EAE
:100F9000FE6F270EFF6FFE07000EFF5B060E0301BC
:100FA000FA5D02E28C8008D00301FE51FF1107E1D7
:100FB0008C708C50010B02E08C9212008C8212001B
:100FC00013EE00F023EE00F0F86A049C4FEC07F0FB
:0C0FD000F5EC07F09EEC07F0FBD71200D8
:040FDC0000EE00F033
:0A0FE0000F0EEE6AEA62FDD7120060
:020FEA001200F3
:020FEC00000003
:020000040030CA
:0100000024DB
:010001000EF0
:010002003FBE
:010003001EDE
:010005008179
:010006008178
:010008000FE8
:01000900C036
:01000A000FE6
:01000B00E014
:01000C000FE4
:01000D0040B2
:00000001FF
